:1000000008308A0000280000FF00030E8301A100D1
:100010000A08A0008A010408A2007708A300780853
:10002000A4007908A5007A08A6007B08A70083131E
:1000300083128C308400801C1F288C1836288B1E5D
:1000400023280B193928220884002308F7002408E4
:10005000F8002508F9002608FA002708FB00200808
:100060008A00210E8300FF0E7F0E09008A110A12FA
:1000700087298A110A126E290A108A100A1182072A
:100080004E34753462346F34743469346334733489
:10009000203455346E34693463346F3464346534D9
:1000A000723420344D3445342D34323431343034CC
:1000B00020344334433453342034433420344434E0
:1000C00065346D346F340D340A3400340A108A10EC
:1000D0000A118207443465346234753467343A3423
:1000E0002034253475340D340A3400340A108A1053
:1000F0000A11820755346E34693463346F346434C2
:1001000065347234203469346E34693474343A346A
:100110000D340A34533479346E3463343A34203431
:1001200000340A108A100A1182070D340A3445344B
:10013000633468346F343A34203400340A108A103F
:100140000A1182074634613469346C34653464348E
:10015000203474346F34203464346534743465343A
:1001600063347434203455346E34693463346F34FA
:100170006434653472342E3420342034483461348D
:100180006C34743469346E3467342E340D340A346C
:1001900000340A108A100A11820747346534743417
:1001A00020347334743461347434753473343A34B1
:1001B00020343034783425346C3478340D340A34B7
:1001C00000340A108A100A118207473465347434E7
:1001D00020346E3461346D3465343A34203425343F
:1001E00073340D340A3400340A108A100A11FB3EAD
:1001F00003188A0A820043346F346E3473347434C3
:1002000061346E34743473340D340A3400340A1497
:100210008A100A118207253464342E342034303495
:10022000783425343034323478340D340A340034A0
:100230000A148A100A1182074D346F346E346934FF
:1002400074346F34723469346E3467342034553406
:100250006E34693463346F346434653472340D340D
:100260000A3400340A148A100A118207543469349B
:100270006D346534203444346934733474346134F7
:100280006E3463346534203441346E3467346C34F6
:1002900065342034563465346C346F3463346934D7
:1002A00074347934203450346534723469346F34A2
:1002B00064340D340A3400340A148A100A11820797
:1002C00025346C34643420342034203420342034F9
:1002D00020342034203420340D340034FF308100A9
:1002E000861D7B290130C1070318C20A0319C30AFE
:1002F0000319C40A8329FF30C107031CC207031C6A
:10030000C307031CC4070B118A110A1223280130EA
:10031000B9070318BA0A0319BB0A0319BC0ABD0AB4
:100320000319BE0A3D08C83C031D9E29BE08031DD3
:100330009E29BF0A0319C00ABE01BD018C108A1193
:100340000A12232852308400831300080319B529A8
:100350000630F800F701F70BAB29F80BAA297B3020
:10036000F700F70BB129800BA82900341B30831646
:100370008500FF308600870088000914891409155C
:1003800081131F149F141F159F1183121F139F1792
:1003900083169F1383121F14831609122F30F70040
:1003A000831281018130840083130008C03907382B
:1003B000800064000008C739F719C039770480004D
:1003C000FF3081001830F80004389200FF308316A7
:1003D00092008C14C03083128B04CB014B083C205C
:1003E000CB0AF70077080C1EF329990025304B0241
:1003F000031DEE290A30D200A2210A30D200A22128
:100400008A150A12572894138C115308930002304E
:10041000941B112A8C1D0A2A00308316111B0130EF
:100420008312F80000341413831691159119162ABB
:1004300077189112771C91161116111A1D2A831222
:100440001308F8000034831611141118252A3030CF
:100450008312D3000322D0012F08500203183A2A36
:1004600029305007840083130008D200D3000322F0
:10047000D00A2C2AB60803198A2A4F08F03C031D1B
:100480004D2AB7080319472A3708D200A22183163C
:1004900091149118492A5C2A831283161115111997
:1004A0004F2A8312B7080319582A3708D200A2210D
:1004B0008316111411185A2A31308312D3000322E3
:1004C000D0010130360250020318792A0730500754
:1004D000F800FA010318FA0A7808293E8400831309
:1004E0007A1883170130F700132278088000D00AA9
:1004F000612A01303602073EF800FA010318FA0AB1
:100500007808293E840083137A188317F701132291
:10051000780880008316111511198C2A8312003473
:100520005308F80152020318982A5208F700A42A27
:10053000F7010830D400D20DF70D530877020318E5
:10054000F700F80DD40B9B2A0034D0015008662028
:10055000D00AF70077080C1EAB2A9900073050022A
:10056000031DA62A4F08D0001B30D1005008D2002E
:100570006430D30090227708D00078083030031D13
:10058000C82AD11CD02AD119D02A511A2030CB2AFE
:10059000D11151125114F80778080C1ECD2A990078
:1005A0005008D2000A30D30090227708D000780893
:1005B0003030031DE12AD119E62A511CE62A511ACE
:1005C0002030F80778080C1EE32A99003030D00755
:1005D00050080C1EE92A99000D300C1EED2A9900D6
:1005E0000A300C1EF12A990000340130CC00CD01F4
:1005F000CE014E087620CE0AF70077080C1EFE2AA0
:10060000990016304E02031DF92ACB014B08093C14
:10061000031C332B2E300C1E0B2B99002E30A900FF
:100620000130AF00B600B701F030CF002322300810
:100630002E3C031D1E2B0130B800232B8130B80047
:100640003808CF00A522CD013808CC004C0B2B2B4D
:10065000CD0803192E2B4C08CF00A5220230D20062
:10066000A221CB0A062B4C0B382BCD0803193D2BAE
:100670004C08F8004D08F900862BCE014E08912059
:10068000CE0AF70077080C1E432B990008304E0263
:10069000031D3E2BCB014B08093C031C7A2B2E304B
:1006A0000C1E502B99004530A9000F30AA000230D3
:1006B000AF00B600B701F030CF0023223108F03C84
:1006C000031D652B0130B8006A2B8730B80038084D
:1006D000CF00A522CD013808CC004C0B722BCD08E1
:1006E0000319752B4C08CF00A5220230D200A2219D
:1006F000CB0A4B2B0D300C1E7B2B99000A300C1EA5
:100700007F2B99004C08F8004D08F9008A150A1251
:100710005A285330A9000130AF000330B600B701AA
:10072000F030CF0023223008533C031D9A2B0130B8
:10073000B8009F2B8830B8003808CF00A522CC0124
:10074000CE013208FA0000303107F8004C080318D7
:100750004C0FFA077A08F9008A150A127728CE1B7F
:10076000C22B0F30F7004D0EF7050A307702031841
:10077000BC2B3030F707BE2B4E08F70777080C1E4E
:10078000BF2B99000F30CD050A304D020318CA2B3C
:100790003030CC2BCE134E08CD074D080C1ECE2B7F
:1007A000990000344330A9000130AF00B600643036
:1007B000B700F030CF0023223008613C031DE32B4B
:1007C0000130B800E82B8530B8003808CF00A522EA
:1007D0008A150A12A3284E30A9000130AF00053057
:1007E000B600B701F030CF00232230084E3C031D85
:1007F000222C0130B8004B08840083134C18831757
:100800003108800001304B07840083134C18831794
:100810003208800002304B07840083134C18831782
:100820003308800003304B07840083134C18831770
:100830003408800004304B07840083134C1883175E
:100840008001272C9530B8003808CF00A522CE01B2
:10085000D0013308FA0000303207F8004E080318C0
:100860004E0FFA077A08F9008A150A12A9284630AD
:10087000A9004B08AA000230AF000330B6000230D6
:10088000B7000F30CF0023223008463C031D4E2C0A
:100890000130B8003208F800552C532C8230B800D3
:1008A0003808CF00A5220030F8008A150A12E62881
:1008B00020304D1E3030CE004C08F700CC1F672C86
:1008C000F709F70A7708CC002D30CE00CD174C0879
:1008D000D2006430D30090227708CC003030780703
:1008E000CF004C08D2000A30D30090223030770776
:1008F000D10030307807D0004E08F700CD1D822C93
:10090000CD1F4D114D1A8F2CCD1FAA2C4D19AA2C7D
:100910007708CF00CD18AA2C7708D000AA2C303049
:100920004F02031DAA2C7708CF002030CE00CD1D2A
:100930009D2C4D11CD14CD1FCD1030305002031D14
:10094000AA2C7708D0002030CF00CD1D9D2CCD10D3
:10095000CD1F4D104D1DB02C4E080C1EAD2C990016
:10096000CD1CB62C4F080C1EB32C99004D1CBC2C72
:1009700050080C1EB92C990051080C1EBD2C990072
:100980008A150A12EF285430A9000130AF00053053
:10099000B600B701F030CF0023223008543C031DCD
:1009A000242D0130B800CE01CD01CC013108CB009F
:1009B000D201D101D0013208CF005108FA0050080D
:1009C000F9004F08F800F7017708CB0778080318FB
:1009D000780FCC0779080318790FCD077A08031828
:1009E0007A0FCE07D201D101D0013308CF005008D1
:1009F000FA004F08F900F701F8017708CB077808EB
:100A00000318780FCC0779080318790FCD077A08F7
:100A100003187A0FCE07D201D101D0013408CF00DC
:100A2000FA00F701F801F9014B08F7074C08031821
:100A30004C0FF8074D0803184D0FF9074E0803181F
:100A40004E0FFA072D2D292D9130B8003808CF0010
:100A5000A522F701F801F901FA018A150A123629CF
:100A60004430A9000130AF000530B600B701F030C6
:100A7000CF0023223008443C031D912D0130B800E3
:100A8000D201D101D0013108CF00D601D501D40166
:100A90003208D3005508FA005408F9005308F8004A
:100AA000F7017708CF0778080318780FD00779087F
:100AB0000318790FD1077A0803187A0FD207D601E5
:100AC000D501D4013308D3005408FA005308F900C3
:100AD000F701F8017708CF0778080318780FD007D7
:100AE00079080318790FD1077A0803187A0FD2070B
:100AF000D601D501D4013408D300FA00F701F8017A
:100B0000F9014F08F70750080318500FF80751086C
:100B10000318510FF90752080318520FFA079A2DBC
:100B2000962D9030B8003808CF00A522F701F801C3
:100B3000F901FA018A150A124129F701F801F901B0
:100B4000FA01E701E801E901EA01660865046404C5
:100B500063040319DB2D2030EB000310DF0DE00DE3
:100B6000E10DE20DE70DE80DE90DEA0D66086A02F8
:100B7000031DC42D65086902031DC42D64086802A5
:100B8000031DC42D63086702031CD52D6308E7020B
:100B90006408031C640FE8026508031C650FE90282
:100BA0006608031C660FEA020314F70DF80DF90D31
:100BB000FA0DEB0BAD2D673084008313003404086D
:100BC000D700D61FF02DD703D716D309D409D509DE
:100BD000D609D30A0319D40A0319D50A0319D60A68
:100BE0003B30DE009A30DD00CA30DC00DB010A3029
:100BF000D9005608E2005508E1005408E000530807
:100C0000DF005E08E6005D08E5005C08E4005B08C4
:100C1000E3009D250008D300840A0008D400840A5C
:100C20000008D500840A0008D600F708031D2B2E03
:100C30005908013A03192B2E570803192D2E0F3985
:100C400059020319252E03184C2ED71B4C2E571B67
:100C50002D2E2030472E2030D705D71E392ED71203
:100C60007708D7002D300C1E332E99005708F70057
:100C7000D7013030D71E472ED7127708D7002D3036
:100C80000C1E402E99005708F700D7013030F707A7
:100C900077080C1E492E99005E08E2005D08E1000D
:100CA0005C08E0005B08DF00E601E501E4010A30D2
:100CB000E3009D257A08DE007908DD007808DC0075
:100CC0007708DB00D90BF92D00345730A90001302B
:100CD000AF000330B600B701F030CF002322300858
:100CE000573C031D872E0130B800CC013108CB00E2
:100CF000CE013208CD00FA0000304B07F8004C0856
:100D000003184C0FFA077A08F9008F2E8C2E8E30BC
:100D1000B8003808CF00A5220030F800F9008A1585
:100D20000A126E295630A9000130AF000330B60018
:100D3000B701F030CF0023223008563C031DB42EFB
:100D40000130B800CE013108CD00D0013208CF000B
:100D5000FA0000304D07F8004E0803184E0FFA074E
:100D60007A08F900BC2EB92E8B30B8003808CF00B5
:100D7000A5220030F800F9008A150A127529D7015A
:100D80000408D6005710831B5714D01FCF2ED61738
:100D9000561ED60ACF09D009CF0A0319D00A500E21
:100DA000F038D200D207E23ED300323ED5005008E0
:100DB0000F39D307D307D507E93ED400D407D407AA
:100DC0004F0E0F39D407D507D40DD50DD509D50D44
:100DD0004F080F39D507D20D0730D1000A30D5079B
:100DE000D403031CEF2ED407D303031CF32ED30725
:100DF000D203031CF72ED207D103031CFB2E513064
:100E00008400831307305605561384035605031DCB
:100E1000102F561A840A561A102F2030F7002D2F43
:100E2000840755300402031956170008F700031D04
:100E3000212F561B212F561A312FD619212F203042
:100E40002C2FD61F292F2D30F70084035613D613CD
:100E50002D2FD61556123030F70777080C1E2E2F7F
:100E60009900840A561F112F00345030A900013018
:100E7000AF000530B600B701F030CF0023223008B4
:100E8000503C031D962F0130B800CE01CD01CC019E
:100E90003108CB00D201D101D0013208CF00510876
:100EA000FA005008F9004F08F800F7017708CB075F
:100EB00078080318780FCC0779080318790FCD0745
:100EC0007A0803187A0FCE07D201D101D001330876
:100ED000CF005008FA004F08F900F701F801770831
:100EE000CB0778080318780FCC0779080318790F17
:100EF000CD077A0803187A0FCE07D201D101D001AD
:100F00003408CF00FA00F701F801F9014B08F707A0
:100F10004C0803184C0FF8074D0803184D0FF9073C
:100F20004E0803184E0FFA079F2F9B2F9430B800DE
:100F30003808CF00A522F701F801F901FA018A1556
:040F40000A129629D2
:1010000003081F3983005730F70020308400831312
:101010008001840AF70B0828F801F901FA01FB01A5
:10102000FC01FD01FE015030F700A0308400831365
:101030008001840AF70B18286030F7001030840014
:1010400083178001840AF70B212883136030F7008F
:101050009030840083178001840AF70B2B288313B8
:10106000A001840183131F3083052030831699006B
:10107000A6309800903083129800A815280883168F
:1010800087008312281628088316870031309300C2
:101090002830831294008316941714131F149F147E
:1010A0001F159F11FF308312A8008A11B6298A15D7
:1010B0008A11F52A8A157908CC007808CB004B0BE9
:1010C0006428CC0803197528CB014B088A119E208F
:1010D0008A15CB0AF70077080C1E6C289900263079
:1010E0004B02031D65287328C2298A11892B8A1592
:1010F0007908CC007808CB00CD014D088A11C920B1
:101100008A15CD0AF70077080C1E842899000E3046
:101110004D02031D7D284C08CD005730CE008A11AA
:10112000AF238A154B08CD005730CE008A11AF236C
:101130008A150D300C1E9A2899000A300C1E9E2824
:1011400099008A11D22B8A15CC014530CB008A1127
:10115000EB2B8A15CB014B088A11E1208A15CB0AAB
:10116000F70077080C1EB22899000A304B02031DC5
:10117000AB28453084008313003000040319C628CF
:1011800000080C1EC1289900840ABC280D300C1ED2
:10119000C72899000A300C1ECB289900CB014B08B8
:1011A0008A11F4208A15CB0AF70077080C1ED6287E
:1011B00099000B304B02031DCF28CA014A080A3C94
:1011C000031C16294A08CB008A11372C8A15780887
:1011D000CB004A08CC001F30CD008A11582C8A154C
:1011E0000230CC004C088A1107218A15CC0AF7007E
:1011F00077080C1EF928990006304C02031DF228CE
:101200004B08CD005730CE008A11AF238A150D3020
:101210000C1E082999000A300C1E0C299900013077
:10122000D2008A11A2218A15CA0ADE28CB014B08F6
:101230008A1118218A15CB0AF70077080C1E1E297F
:10124000990015304B02031D1729CB014B088A1159
:1012500032218A15CB0AF70077080C1E2D29990038
:1012600025304B02031D26298A11C32C8A157A08C2
:10127000CE007908CD007808CC007708CB008A1121
:10128000302D8A157A08D2007908D1007808D0006C
:101290007708CF00413084004E08D6004D08D500B5
:1012A0004C08D4004B08D3008A11DF258A15203062
:1012B0000C1E58299900413084005208D60051086C
:1012C000D5005008D4004F08D3008A11DF258A15B5
:1012D00020300C1E692999008A11652E8A1579081B
:1012E000CC007808CB008A11922E8A157908CE009E
:1012F0007808CD00103084004C08D0004B08CF0097
:101300008A11BF268A1520300C1E842999001030BE
:1013100084004E08D0004D08CF008A11BF268A15E0
:1013200020300C1E912999008A11352F8A157A08D0
:10133000CE007908CD007808CC007708CB0041308A
:1013400084004E08D6004D08D5004C08D4004B0848
:10135000D3008A11DF258A150330CF004F088A1188
:101360005C218A15CF0AF70077080C1EB529990071
:101370000D304F02031DAE296430D2008A11A22124
:061380008A153429630008
:02400E00323F3F
:00000001FF
